:020000040800F2
:1000000018800020690200083930000845290008DE
:1000100025300008050B0008B93F0008000000006B
:100020000000000000000000000000004939000846
:10003000E51F0008000000009D310008A13A0008FB
:10004000830200088302000883020008830200087C
:10005000830200088302000883020008830200086C
:1000600085200008B5200008C92000088302000888
:10007000830200088302000883020008830200084C
:10008000830200088302000883020008830200083C
:10009000830200088302000883020008F920000898
:1000A000830200088302000883020008830200081C
:1000B000830200080D3B0008830200088302000849
:1000C00083020008830200088302000883020008FC
:1000D00083020008830200088302000883020008EC
:1000E000E91F000883020008830200088302000859
:1000F00083020008830200088302000883020008CC
:1001000083020008830200088302000883020008BB
:1001100083020008830200088302000883020008AB
:10012000830200088302000883020008830200089B
:10013000830200088302000883020008830200088B
:10014000830200088302000883020008830200087B
:10015000830200088302000883020008493C00086B
:10016000830200088302000883020008830200085B
:10017000830200088302000883020008830200084B
:10018000830200088302000800F002F800F05CF827
:100190000AA090E8000C82448344AAF10107DA45E2
:1001A00001D100F051F8AFF2090EBAE80F0013F0D8
:1001B000010F18BFFB1A43F0010318472841000044
:1001C000484100000A444FF0000C10F8013B13F0C6
:1001D000070408BF10F8014B1D1108BF10F8015BA0
:1001E000641E05D010F8016B641E01F8016BF9D193
:1001F00013F0080F1EBF10F8014BAD1C0C1B09D1EA
:100200006D1E58BF01F801CBFAD505E014F8016B5B
:1002100001F8016B6D1EF9D59142D6D370470000ED
:100220000023002400250026103A28BF78C1FBD8FF
:10023000520728BF30C148BF0B6070471FB504F09C
:100240004BF81FBD10B510BD00F018F91146FFF7AF
:10025000F5FF03F063FF00F036F903B4FFF7F2FF98
:1002600003BC00F03DF900000948804709480047F9
:10027000FEE7FEE7FEE7FEE7FEE7FEE7FEE7FEE756
:10028000FEE7FEE704480549054A064B70470000B3
:10029000A53A000889010008186000201880002095
:1002A000187000201870002010B5431C02E010F8F0
:1002B000011B71B18107FAD14FF0013202C88C1ACB
:1002C0008C4314EAC211F9D0C01A0A0603D0C01E2A
:1002D00010BDC01A10BD0A0401D0801E10BD090255
:1002E000FCD0401E10BD032A40F2308010F0030CF9
:1002F00000F0158011F8013BBCF1020F624498BF79
:1003000011F801CB00F8013B38BF11F8013BA2F115
:10031000040298BF00F801CB38BF00F8013B11F090
:10032000030300F05280083AC0F0088051F8043B03
:10033000083A51F804CBA0E80810F5E7121D5CBF9D
:1003400051F8043B40F8043BAFF30080D20724BFD0
:1003500011F8013B11F801CB48BF11F8012B24BF64
:1003600000F8013B00F801CB48BF00F8012B7047B3
:1003700002F0FF0343EA032242EA024200F002B81D
:100380004FF000020429C0F0128010F0030C00F0BE
:100390005080CCF1040CBCF1020F18BF00F8012B07
:1003A000A8BF20F8022BA1EB0C0100F042B85FEAD5
:1003B000C17C24BF00F8012B00F8012B48BF00F8D6
:1003C000012B704770477047704710B5203AC0F056
:1003D0000B80B1E81850203AA0E81850B1E8185046
:1003E000A0E81850BFF4F5AF5FEA027C24BFB1E883
:1003F0001850A0E8185044BF18C918C0BDE81040F4
:100400005FEA827C24BF51F8043B40F8043B08BFFC
:100410007047D20728BF31F8023B48BF11F8012BC3
:1004200028BF20F8023B48BF00F8012B70474FF06F
:10043000000200B5134694469646203922BFA0E834
:100440000C50A0E80C50B1F12001BFF4F7AF090740
:1004500028BFA0E80C5048BF0CC05DF804EB890031
:1004600028BF40F8042B08BF704748BF20F8022B74
:1004700011F0804F18BF00F8012B7047754600F04F
:100480002BF8AE4605006946534620F00700854626
:1004900018B020B5FFF7F6FEBDE820404FF000068B
:1004A0004FF000074FF000084FF0000B21F007015C
:1004B000AC46ACE8C009ACE8C009ACE8C009ACE89F
:1004C000C0098D46704710B50446AFF30080204642
:1004D000BDE81040FFF7C1BE00487047B45F002080
:1004E00001491820ABBEFEE726000200704770B538
:1004F00006460C46154608E03046721C96B200F0DF
:1005000007F804F8010B681E85B2002DF4D170BD08
:100510002DE9F04104460025002702F087FCA020C9
:1005200002F050FC02F0D4FC054605B129E020128F
:1005300002F048FC02F0CCFC054605B121E026465D
:10054000E11704EB11610912A4EB0121C8B202F01A
:1005500039FC02F0BDFC054605B112E002F066FC74
:10056000A12002F02FFC02F0B3FC054605B108E023
:10057000002002F0F1FB074602F07EFC3846BDE8A1
:10058000F08102F079FC0020F9E72DE9F041054601
:100590000C46164600270CE02178284600F010F89B
:1005A0000746012F02D00020BDE8F081681C85B20B
:1005B000641C301EA6F101018EB2EDD10120F3E7DB
:1005C0002DE9F04104460E46002702F02FFCA02042
:1005D00002F0F8FB02F07CFC0746201202F0F2FB6E
:1005E00002F076FC07462546E11704EB116109127B
:1005F000A4EB0121C8B202F0E5FB02F069FC07465A
:10060000304602F0DFFB02F063FC074602F034FCE8
:100610000F2003F0F1FC0120BDE8F0811CB502F0D1
:1006200045FB01211F2003F049F80620009001201E
:100630008DF8040000208DF8060003208DF80500D9
:1006400001208DF8070069462A4801F0DAFF4FF4CF
:10065000604000906946284801F0D3FF4FF4E05015
:1006600000906946254801F0CCFF43F60100009058
:100670006946234801F0C5FF41F210000090694629
:10068000204801F0BEFF04211A4802F030F84FF470
:100690000051194802F02BF80121194802F027F8FF
:1006A0004FF48051164802F022F84FF4805115485B
:1006B00002F01DF802210F4802F019F8102111482C
:1006C00002F015F8022010490860012100F01CFA20
:1006D0000421002000F018FA47F6FF7001F00CFE2C
:1006E00047F6FF7001F01EFE00F0C0F802F0D0F9EE
:1006F0001CBD00000000024000040240000802404F
:10070000000C0240001002408C0000201CB50121AA
:10071000102002F0D3FF0420009001208DF8040087
:1007200000208DF8060003208DF8050001208DF8CB
:1007300007006946034801F064FF012002F098F9C0
:100740001CBD00000010024010B500244048007895
:10075000012819D13F48006820F0FF003D4908609A
:100760003D484078096808433A49086001213B4800
:10077000007800F0C9F904213648006800F0C4F997
:1007800000203349087001243548007801281AD127
:100790003048006820F47F402E4908602E48407899
:1007A000096841EA00202B49086001212B480078A4
:1007B00000F0AAF904212748006800F0A5F90020FC
:1007C0002749087001242748007801281AD12148B8
:1007D000006820F47F001F4908601F4840780968BE
:1007E00041EA00401B49086001211C48007800F0E4
:1007F0008BF904211748006800F086F90020194998
:10080000087001241848007801281AD1114800689E
:1008100020F07F400F4908600F484078096841EA9E
:1008200000600C49086001210C48007800F06CF968
:1008300004210848006800F067F900200A490870A0
:100840000124012C02D1642003F0F6FB10BD00004E
:100850009000002098000020030100209400002058
:1008600091000020920000209300002000B585B088
:100870000820009000208DF8040003208DF805006A
:1008800002208DF807006946334801F0BAFE4FF4A4
:10089000006000906946314801F0B3FE4FF480706B
:1008A000009069462E4801F0ACFE20200090694679
:1008B0002C4801F0A6FE0121880302F00FFF0B2156
:1008C000022003F043F80821032003F03FF803213E
:1008D000002003F03BF80521042003F037F840F630
:1008E0002810029000208DF80C0008208DF80D00D3
:1008F00001208DF80E0002A801F0B4FC09208DF84B
:10090000100001208DF8110000208DF81200012048
:100910008DF8130004A802F091FB17208DF8100049
:1009200001208DF811008DF812008DF8130004A835
:1009300002F084FB28208DF8100001208DF81100B2
:1009400003208DF8120001208DF8130004A802F096
:1009500075FB05B000BD0000000002400008024029
:10096000000C0240001002402DE9FF5F05460C46D6
:100970002F78EE782879697900EB01201FFA80F84A
:10098000A879E97900EB01201FFA80F98DF8086059
:100990008DF80B40ADF8098001208DF80C0001AAFC
:1009A000DDE9020101F082FF83469DF804105846FC
:1009B00000F06CFF8DF808608DF80B40ADF80990E1
:1009C00000208DF80C00012C00D100BF022C00D1BA
:1009D00000BF6A46DDE9020101F068FF82469DF82A
:1009E0000000032802DB9DF8000000909DF8001035
:1009F000504600F04BFF22463946022001F01CFA17
:100A0000BDE8FF9F0146132901DA00207047A1F1DC
:100A100009000A2290FBF2F302FB130008B1002048
:100A2000F4E70120F2E700002DE9FE4F04460D46F1
:100A3000277894F8018094F8029094F803A0207A23
:100A4000617A00EB01201FFA80FB002000908DF8F6
:100A50000880ADF804B08DF809908DF807708DF816
:100A600006A0012D00D100BF6A46DDE9010101F0B9
:100A700041FE06460EB9BDE8FE8F681EC100009813
:100A8000884005490968084303490860042D00D1DE
:100A900000BF00BFEFE70000880000202DE9F04113
:100AA00005462F781548006800F00040134908609B
:100AB0000026002410E047FA04F000F0010050B1D5
:100AC000621CD1B206EB86036A1C02EB4300FFF7FF
:100AD000ABFF701CC6B2641C042CECDB012108487F
:100AE000006800F011F804210448006800F00CF8D8
:100AF000022003F081FABDE8F081000088000020A8
:100B00008C00002000BFFEE72DE9F04104460E46B0
:100B100000250027012E2BD100BF26E004F080071E
:100B200047B14FF48051324801F0E1FD012003F05C
:100B300083FA07E04FF480512D4801F0D6FD0120E3
:100B400003F07AFA4FF480412A4801F0D0FD0120E9
:100B500003F072FA4FF48041264801F0C6FD0120EF
:100B600003F06AFA6400681CC5B2082DD6DB3CE0CD
:100B7000042E3AD1002526E004F0004747B14FF497
:100B800080511B4801F0B3FD012003F055FA07E046
:100B90004FF48051164801F0A8FD012003F04CFAF3
:100BA0004FF48041134801F0A2FD012003F044FA04
:100BB0004FF480410F4801F098FD012003F03CFA0A
:100BC0006400681CC5B2202DD6DB4FF400410948F3
:100BD00001F08DFD012003F02FFA4FF4004105488C
:100BE00001F083FD012003F027FABDE8F081000049
:100BF00000080240000402402DE9F04106460F467D
:100C000090461C4601257720044908702246294653
:100C1000012003F0EBF8BDE8F0810000B8460020A9
:100C20002DE9F05F81468A4693461E468127394664
:100C30003448FFF7A5FB01F081FE044620783149D6
:100C4000087060784870A0788870002005E0211D49
:100C50000A5CC11C2B4B5A54401C0E28F7DB04F1D4
:100C60001200FFF721FB0546102D01DD102000E0EA
:100C700028460546002007E004F112010A5C00F155
:100C80001101204B5A54401CA842F5DB04F122000C
:100C9000FFF70AFB0546202D01DD202000E0284655
:100CA0000546002007E004F122010A5C00F1210161
:100CB000144B5A54401CA842F5DB04F14200FFF7E4
:100CC000F3FA0546402D01DD402000E028460546A8
:100CD000002007E004F142010A5C00F14101094BE8
:100CE0005A54401CA842F5DB074B3A4605490320FD
:100CF00000F0FCFC804632463946022003F076F8CC
:100D0000BDE8F09FB8460020B84E00202DE9F04F16
:100D1000A9B081468A4693461E4681273946364801
:100D2000FFF72EFB684603F0D3F96C462078324972
:100D3000087060784870A0788870002005E0211D58
:100D40000A5CC11C2C4B5A54401C0E28F7DB04F1E2
:100D50001200FFF7A9FA0546102D01DD102000E072
:100D600028460546002007E004F112010A5C00F164
:100D70001101214B5A54401CA842F5DB04F122001A
:100D8000FFF792FA0546202D01DD202000E02846DD
:100D90000546002007E004F122010A5C00F1210170
:100DA000154B5A54401CA842F5DB04F14200FFF7F2
:100DB0007BFA0546402D01DD402000E0284605462F
:100DC000002007E004F142010A5C00F141010A4BF6
:100DD0005A54401CA842F5DB084B3A46064903200A
:100DE00000F084FC804632463946032002F0FEFFC4
:100DF00029B0BDE8F08F0000B8460020B84E0020B2
:100E00002DE9F041AAB006460F4690461C460E2535
:100E100001A803F05DF92A460DF18E010548FFF7A0
:100E200062FA22462946042002F0E0FF2AB0BDE81B
:100E3000F0810000B846002003F05EF9012080F345
:100E4000138800BF00BFBFF34F8F0748006800F44E
:100E5000E06006490843001D03490860BFF34F8F57
:100E600000BF00BFFEE700000CED00E00000FA0547
:100E70002DE9F04105460C461646984627465EB1D8
:100E80002146284601F09AFD08B9BDE8F0812046C8
:100E900004EBD071C1F34F07142F07DA002003E0F1
:100EA000295C034A1154401CB842F9DB00BFECE74F
:100EB000240100202DE9F04106460F4690461C46CD
:100EC00014252A4605490648FFF70DFA2246294609
:100ED000072002F08BFFBDE8F08100002401002014
:100EE000B84600202DE9F043A9B005460C46164649
:100EF0009946012704F0FF0856B1204604EBD07153
:100F0000C1F347082146284601F058FD00B90027E3
:100F1000B8F10E0F00DA002767B1684603F0D8F881
:100F20000E2229460DF18A00FFF7DDF9684603F02D
:100F3000D9F803E00121022000F08CFC29B0BDE8C3
:100F4000F0832DE9F04104460D4616461F46012167
:100F5000902000F07FFCBDE8F08170472DE9FF4F45
:100F600085B004460E464248007810B109B0BDE88D
:100F7000F08F01203E490870324621463D48FFF778
:100F8000B2F93046FFF73EFD38B900203849087005
:100F90000121052000F05EFCE8E7A6F10800C5B2DB
:100FA000281D00F0FF08615D681C205C01EB00213A
:100FB000A81C205C01EB0041E81C205C01EB0060F8
:100FC000049014F8081008F10100205C01EB0020E7
:100FD0001FFA80FB2946204601F0DAFC03902946DF
:100FE000204601F038FD8146DDE90310884201D139
:100FF000CB4507D000201E4908700121FF2000F0DA
:1010000029FCB3E74FF0000A207802902046FFF752
:1010100045FD002712E00298384100F0010060B160
:101020007A1CD1B20AEB8A03621C02EB4300FFF781
:101030009BFC0AF1010000F0FF0A7F1C042FEADB91
:1010400002200190002006E0B11E0144615C0A4AC2
:101050001154411CC8B20228F6DB2220089A0199DB
:1010600002F0C4FE00200249087000BF7EE70000C5
:1010700084000020805F0020B84600202DE9F04762
:101080000546884691469A464A464146284601F01A
:10109000AFF928B90121052000F0DCFBBDE8F0879D
:1010A0002F78002600240FE047FA04F000F001003A
:1010B00048B1621CD1B206EBC6036A1C981801F055
:1010C00047F9701CC6B2641C042CEDDB00BFE5E7D9
:1010D0002DE9F0470546884691469A462E78002726
:1010E000002420E046FA04F000F00100D0B1012015
:1010F00000EB8400285C00F00101022000EB84007A
:10110000285C61F35F10074632463946042000F040
:1011100093FE042000EB84002F5C32463946052004
:1011200000F08AFE641C042CDCDB00F0A1FBBDE8AF
:10113000F08700002DE9F0478046894692461D461B
:1011400008261348008884B2200A124908704C709F
:101150001148008884B2200A8870CC700F4800883B
:1011600084B2200A08714C710D48008884B2200AAC
:101170008871CC710B4B3246302000F0B7FA07462D
:101180002A463146302002F031FEBDE8F0870000EB
:10119000BC000020B8460020BE000020C000002097
:1011A000C2000020B84E00202DE9F04105460E4651
:1011B00017461C462146012002F0CEFCBDE8F08116
:1011C0002DE9F04104460D4616461F4601219020A8
:1011D00000F040FBBDE8F0812DE9F05F07460C46CA
:1011E00015461E464FF0010804F0FF095DB1204688
:1011F00004EBD071C1F347092146384601F0DEFB0C
:1012000008B94FF00008B9F1010F01D04FF0000804
:10121000B8F1000F05D10121052000F01BFBBDE84E
:10122000F09F4FF0640A0749384601F0B8FF824644
:1012300001F089FF834632465146332002F0D6FD45
:1012400000BFECE7B84600202DE9F04104460E4609
:101250001546984601272B463A463146204601F06E
:10126000D0FB28B90121022000F0F4FABDE8F0819A
:10127000207802F0F1F900BFF8E700002DE9F05FF7
:1012800006460C4617469B464FF0010804F0FF093E
:101290005FB1204604EBD071C1F3470921463046C7
:1012A00001F08CFB08B94FF00008B9F1050F01DA25
:1012B0004FF00008B8F1000F17D096F800A00120F9
:1012C0000D49087000250DE04AFA05F000F0010014
:1012D00038B1681CC1B2701C00F0E0F90A2002F0BD
:1012E000ABFE6D1C042DEFDB03E00121052000F0B7
:1012F000B1FABDE8F09F0000840000202DE9F05F06
:1013000006460C4617469B464FF0010904F0FF0ABB
:101310005FB1204604EBD071C1F3470A2146304645
:1013200001F04CFB08B94FF00009BAF1050F01DAE2
:101330004FF00009B9F1000F1ED0012004E0315C2C
:1013400001EB0828411CC8B20528F8DB3078801F63
:10135000C5B225B90121404600F086FB05E0012D0C
:1013600003D10221404600F07FFB022D03D103216F
:10137000404600F079FB03E00121052000F06AFA05
:10138000BDE8F09F2DE9F05F06460D4617469B46E7
:101390004FF0010905F0FF0A5FB1284605EBD07157
:1013A000C1F3470A2946304601F008FB08B94FF05F
:1013B0000009BAF1020F01DA4FF00009B9F1000F8C
:1013C00005D10121052000F045FABDE8F09F96F80F
:1013D00001803478012C05D101224146022000F021
:1013E0002BFD16E0022C05D102224146104600F0EA
:1013F00023FD0EE0042C05D103224146022000F01B
:101400001BFD06E0082C04D104224146022000F016
:1014100013FD142002F010FE00BFD6E72DE9F047BF
:1014200004468846174699463B46062241462046D2
:1014300001F0E7FA28B90121052000F00BFABDE818
:10144000F0876078217800EB01260025022004E077
:10145000215C01EB0525411CC8B20628F8DB0749D1
:101460000E700748056001213046FFF74DFB04214F
:101470002846FFF749FB00BFE1E700009400002089
:10148000980000202DE9F04105460E4614461F46FF
:10149000234612223146284601F0B3FA28B9012129
:1014A000052000F0D7F9BDE8F0811221284601F0AF
:1014B00045FD00BFF7E700002DE9F0479AB006466A
:1014C0000C4617469A464FF0010804F0FF094FB149
:1014D000204604EBD071C1F347092146304601F0A4
:1014E0006DFA8046B9F1070F01DA4FF00008B8F144
:1014F000000F06D10121052000F0ACF91AB0BDE8BB
:10150000F0871648007800B1F8E701201349087009
:10151000652C0ADA002004E0FF2122180DF80210E1
:10152000401CC4F165018142F6DC22463146684622
:10153000FEF7D9FE0DF10101684601F085FE054672
:10154000012D02D100F094F903E00121FF2000F009
:1015500081F900200149087000BFCFE78400002016
:101560002DE9F04104460D4616461F4602F042FBA7
:10157000BDE8F081F8B504460D4616461F4600F05A
:1015800077F902F02DFE00200090F8BD00F070F910
:1015900000BFFEE72DE9F04705460C461746984682
:1015A0004FF0010904F0FF0A5FB1204604EBD0714F
:1015B000C1F3470A2146284601F000FA08B94FF066
:1015C0000009BAF1020F01DA4FF00009B9F1000F7A
:1015D00005D10121052000F03DF9BDE8F087022684
:1015E000287820B1012804D0022806D103E029265A
:1015F00004E0082602E0082600E000BF00BF06F174
:101600000801FF221448FEF7B3FE287820B1012814
:1016100008D0022816D10DE0312210490E48FEF7FD
:1016200062FE10E00C480E49096801600D49096826
:10163000416008E008480C49096801600B490968E5
:10164000416000E000BF00BF42463146E32002F0A7
:10165000CDFB00BFC1E70000B8460020805F00203E
:101660001C01002020010020AC020020A802002064
:101670002DE9F04104460F4690461D468026802203
:1016800021460548FEF72FFE2A463146E42002F0A7
:10169000ADFBBDE8F0810000B84600202DE9FE4317
:1016A00004460D4626786778A078E17800EB0120A3
:1016B0001FFA80F80EB9012600E000268DF80070B0
:1016C0008DF80350ADF801808DF8046002AADDE9C1
:1016D000000101F0EBF881469DF80810484600F043
:1016E000D5F8012002F088FCBDE8FE832DE9F04129
:1016F00006460F4615461C4655202070AA206070ED
:10170000BB20A070E6702571280A6071002D04DDF1
:101710002A463946A01DFEF7E6FD0D21A81D2154DD
:101720000A21E81D2154401CBDE8F0812DE9F0415B
:101730003A483B49098830F811504FF6FF7085420E
:1017400001D1BDE8F0814FF6FF703449344A128868
:1017500021F8120000200CE03249495D324A115450
:10176000691C44F2080291FBF2F302FB13118DB2E3
:10177000401CB0F5026FEFDB2B480078552807D1ED
:1017800029484078AA2803D127488078BB2800D070
:10179000D7E7254EB088801D3146085C0D2804D15E
:1017A000B088C01D085C0A2800D0CAE71B481C4945
:1017B000098830F811501A480088401C142190FB09
:1017C000F1F201FB120016490880174F002420E0B7
:1017D00004EB4400154911F82000F978884216D12D
:1017E00004EB4400DFF8448008EB8000437A04EB0C
:1017F000440008EB8000027AB98804EB440008EB4F
:101800008000D0F804C00848801DE04703E0601C59
:10181000C4B21E2CDCDB00BF00BF92E738570020AB
:1018200018010020B0060020605700203801002079
:1018300070B514240125224604490548FEF753FDDE
:101840002A462146072002F0D1FA70BD240100206B
:10185000B846002070B504460D46012603480470C2
:101860002A463146B02002F0C1FA70BDB8460020C9
:1018700010B50224C0200449087048700122214696
:1018800002F0B4FA10BD0000B84600202DE9F04780
:1018900004460E460027B8460025A946012E04D06E
:1018A000022E19D0032E48D130E001216B4800F000
:1018B0001CFF012002F0C0FB0121684800F017FF67
:1018C000012002F0B9FB0121644800F00EFF012065
:1018D00002F0B2FB012531E04FF40051604800F006
:1018E00004FF012002F0A8FB4FF400515C4800F017
:1018F000FEFE012002F0A0FB4FF40051584800F01A
:10190000F4FE012002F098FB022517E0042155485F
:1019100000F0EBFE012002F08FFB0421514800F0A3
:10192000E6FE012002F088FB04214E4800F0DDFEB7
:10193000012002F081FB032500E000BF00BF4FF44F
:10194000C051474800F0D3FE012002F075FB4FF470
:101950000061434800F0C9FE012002F06DFB4FF426
:1019600080513F4800F0C1FE012002F065FB0027D6
:101970004AE04FF000082AE004F00049B9F1000FF6
:1019800008D04FF40061364800F0B1FE012002F0AB
:1019900053FB07E04FF40061314800F0A6FE012040
:1019A00002F04AFB4FF480512D4800F0A0FE0120C8
:1019B00002F042FB4FF48051294800F096FE0220CD
:1019C00002F03AFB640008F1010000F0FF08B8F1F2
:1019D000080FD1DB4FF40061214800F086FE0120A2
:1019E00002F02AFB4FF480511D4800F080FE0120D8
:1019F00002F022FB4FF48051194800F076FE0220DD
:101A000002F01AFB781CC7B2042FB2DB4FF48051EE
:101A1000134800F06CFE012002F00EFB4FF4006151
:101A20000F4800F064FE012002F006FB012D03D1F7
:101A300001210A4800F05BFE022D03D1290308486A
:101A400000F055FE032D03D10421064800F04FFE9F
:101A5000012002F0F1FA0025BDE8F087000C0240F9
:101A600000040240000002402DE9F04704460D4604
:101A70000027C4F3034848F03009A6B2012D04D072
:101A8000022D04D0032D06D103E0182705E01A2704
:101A900003E01C2701E0BDE8F08700BF01F062F819
:101AA000384601F02BF801F0A9F800B149E04846AA
:101AB00001F024F801F0A2F800B142E0300A01F090
:101AC0001DF801F09BF800B13BE0F0B201F016F810
:101AD00001F094F800B134E001F06AF8012D04D06F
:101AE000022D0ED0032D26D119E00121174800F058
:101AF000FCFD052002F0A0FA0121144800F0F7FDDA
:101B00001AE04FF40051124800F0EFFD052002F0FA
:101B100093FA4FF400510E4800F0E9FD0CE0042167
:101B20000C4800F0E2FD052002F086FA0421094885
:101B300000F0DDFD00E0AEE700BF012002F05CFA3E
:101B4000A9E701F035F800BFA5E70000000C02404E
:101B5000000402400000024010B500241448006850
:101B600020F440101249086008460068086004E04C
:101B7000601CC4B2012002F05FFA0E48006808B190
:101B8000C82CF5DBC82C01DB012010BD002404E0CB
:101B9000601CC4B2012002F04FFA0648006808B980
:101BA000F02CF5DBF02C01DB0120EEE70020ECE768
:101BB000000802402802414210B5002400F0B0F8AD
:101BC00000F08CF8FFF7C8FFCC2000F0B5F8BE207D
:101BD00000F0B2F800F03CF804B2200104B2204654
:101BE000E11704EB11710C1101480480204610BD6F
:101BF000BC0000201CB540F20140009001208DF88F
:101C0000040000208DF8060002208DF80500012058
:101C10008DF8070069460B4800F0F3FC4FF40070A4
:101C200000906946084800F0ECFC4FF4007000900A
:101C30006946064800F0E5FC00F050F8FFF78CFF1D
:101C40001CBD000000080240000C024000100240D1
:101C500070B50026002408E000F00CF8054605FAEF
:101C600004F0304386B2601CC4B20C2CF4DB304666
:101C700070BD000010B500241548006820F4401025
:101C8000134908600846006840F48010086000208E
:101C900010490860022002F0CFF901200E49C1F876
:101CA000A8020B48006820F4401009490860084663
:101CB000006808600C2002F0BFF906488038006810
:101CC00000B10124322002F0B7F9204610BD000017
:101CD00000080240A80241420000414210B50D48F0
:101CE000006820F440100B4908600846006840F482
:101CF0008010086000200849086040F2EE2002F0E1
:101D00009BF901200549C1F8A8020F2002F094F9BF
:101D100010BD000000080240A802414200004142FC
:101D200010B5FFF7DBFFFFF717FFCC2000F004F83A
:101D3000442000F001F810BD70B504463648006834
:101D400020F44010344908600846006840F48010D0
:101D500008603248006820F4402030490860084696
:101D6000006840F4802008602D48006820F440207E
:101D70002B4908600846006840F480200860264827
:101D8000006820F00300244908600846006840F01D
:101D90000100086001253CE004F001066410DEB19A
:101DA0000020204908602049C1F8A4021F490860AA
:101DB0001F49C1F88002022002F03EF901201949B2
:101DC00008601C490860194908601949C1F8800277
:101DD0003C2002F031F91AE0002012490860124953
:101DE000C1F8A402114908601149C1F880023C20E1
:101DF00002F022F901200B4908600E4908600B49E6
:101E000008600B49C1F88002022002F015F9681C35
:101E1000C5B2082DC0DD70BD00080240000C0240B4
:101E200000100240A802414200804142A402424206
:101E300000004142A48241422DE9F04707460E4688
:101E4000904600250024B946B8F1010F09D0B8F139
:101E5000020F0DD0B8F1030F11D0B8F1040F1AD151
:101E600013E04FF480515C4800F041FC012413E082
:101E70004FF48051594800F03AFC03240CE0022151
:101E8000574800F034FC052406E01021534800F0C8
:101E90002EFC062400E000BF00BF022002F0CCF8B8
:101EA000012C04D121034C4800F01FFC14E0032C4A
:101EB00005D14FF48051494800F017FC0CE0052C87
:101EC00004D10221464800F010FC05E0062C03D1A5
:101ED0001021424800F009FC022002F0ADF8002574
:101EE0002BE009F0800ABAF1800F08D14FF40061AD
:101EF000394800F0FCFB022002F09EF807E04FF4A6
:101F00000061354800F0F1FB022002F095F84FF433
:101F10000051314800F0EBFB022002F08DF84FF445
:101F200000512D4800F0E1FB022002F085F84FEA55
:101F300049604FEA1069681CC5B2082DD1DB002545
:101F400029E006F0800ABAF1800F08D14FF4006151
:101F5000214800F0CCFB022002F06EF807E04FF4BD
:101F600000611D4800F0C1FB022002F065F84FF44B
:101F70000051194800F0BBFB022002F05DF84FF45D
:101F80000051154800F0B1FB022002F055F8700630
:101F9000060E681CC5B2082DD3DB012C03D121032A
:101FA0000D4800F0A4FB032C04D14FF480510B48E2
:101FB00000F09DFB052C03D10221094800F097FB9E
:101FC000062C03D11021054800F091FB022002F0FD
:101FD00033F8BDE8F0870000000C0240001002401A
:101FE000000002407047000010B54FF4806000F020
:101FF0002DF9012814D1142001F0FEFF4FF4004107
:102000001B4800F069FB30B91A480078012802D15A
:102010000020184908704FF4806000F011F925E0A5
:102020004FF4805000F012F9012814D1142001F06F
:10203000E3FF4FF48051104800F04EFB30B90F48D9
:102040000078012802D100200C4908704FF480501C
:1020500000F0F6F80AE04FF4006000F0F7F801280D
:1020600004D107490870C00200F0EAF810BD000072
:10207000000C0240A900002000000240A80000203F
:102080009000002010B5142001F0B6FF042107488D
:1020900000F022FB30B906480078012802D1002068
:1020A00003490870042000F0CBF810BD000C02407A
:1020B000A700002010B5012002490870082000F098
:1020C000BFF810BD9200002010B5142001F094FF5D
:1020D0001021074800F000FB30B9064800780128BD
:1020E00002D1002003490870102000F0A9F810BDAB
:1020F000000C0240A600002010B5402000F0A6F819
:10210000012812D1142001F077FF4021124800F07D
:10211000E3FA30B911480078012802D100200F49B4
:102120000870402000F08CF815E0202000F08EF8B8
:10213000012805D10A490870202000F081F80AE042
:102140004FF4807000F082F8012804D1054908702E
:10215000000200F075F810BD000C0240A500002040
:1021600093000020910000200EB50121880301F0AA
:10217000B5FA0221032001F0E9FB0421032001F05C
:10218000E5FB0621032001F0E1FB0821032001F01B
:10219000DDFB0A21002001F0D9FB0C21002001F019
:1021A000D5FB0521042001F0D1FB41F274500090D1
:1021B00000208DF8040008208DF8050001208DF81E
:1021C0000600684600F04EF808208DF8080001204F
:1021D0008DF8090002208DF80A0001208DF80B000F
:1021E00002A800F02BFF0A208DF8080002208DF8CD
:1021F000090001208DF80A008DF80B0002A800F0FC
:102200001DFF28208DF8080003208DF8090002200A
:102210008DF80A0001208DF80B0002A800F00EFFD7
:1022200017208DF8080004208DF8090002208DF891
:102230000A0001208DF80B0002A800F0FFFE0EBD81
:102240000149086070470000143C0140014600202D
:10225000034A12680A400AB1012000E000207047DA
:10226000143C0140002123498279002A3AD00A46D1
:10227000126803689A430B461A600A1D12680368C5
:102280009A430B1D1A60027911440A6803681A43C5
:102290000A60184A0832126803689A43154B0833DB
:1022A0001A601A1D126803689A43124B0C331A60A5
:1022B0004279102A0ED11A1F126803681A430D4B77
:1022C00008331A601A1D126803681A43094B0C334D
:1022D0001A600DE00749427911440A6803681A43FD
:1022E0000A6005E0027911440A6803689A430A60AB
:1022F00070470000003C01402DE9F04105460226F0
:102300000C274FF00108064C44EA076444EA0844ED
:102310002C4331462046FFF7B9FABDE8F0810000B2
:10232000000030102DE9F041054602260C274FF041
:102330000308064C44EA076444EA08442C43314647
:102340002046FFF7A3FABDE8F0810000000030103E
:102350002DE9FF5F04466578A678E77894F8088051
:102360002079617900EB01201FFA80F9A079E179E9
:1023700000EB01201FFA80FA00201B4908601B486F
:1023800000680190002000908DF80C508DF80D60D1
:102390008DF80A708DF80E806B4601AADDE9020106
:1023A00000F03CFA8346BBF1000F01D1BDE8FF9F6E
:1023B0009DF800000C4908600C4901980860012153
:1023C00009480068FEF7A0FB042108480068FEF7F2
:1023D0009BFB4846FFF7A6FF5046FFF78DFF022004
:1023E00001F00AFE00BFE1E78C0000208800002019
:1023F0002DE9F04106460D4617460A2D02DA002067
:10240000BDE8F0810024002009E0012181403278FC
:102410001140012901D1611CCCB2411CC8B2042871
:10242000F3DB681E04EBC401884201D00020E7E71B
:102430004FB104EBC400401C00F0FF084146304699
:1024400000F0BCFADCE70120DAE70000014908608F
:10245000704700000C3C024030B10749096841F464
:102460008061054A116005E00349096821F4806133
:10247000014A116070470000003C024070B50446FC
:102480000A460026092502B909E0012A01D11602EF
:1024900005E0022A01D1160201E04FF4407600F077
:1024A0009FF80546092D28D11548006820F4407092
:1024B0001349086008460068304308600846006811
:1024C00020F0F80008600846006844F00201084364
:1024D0000B4908600846006840F48030086000F04E
:1024E0007FF805460648006820F0020004490860AD
:1024F0000846006820F0F8000860284670BD00001B
:10250000103C024009201349096801F48031B1F5FB
:10251000803F01D101201CE00E49096801F0100143
:1025200009B1062015E00B49096801F4807109B171
:1025300002200EE00749096801F0EF0109B1072008
:1025400007E00449096801F0020109B1082000E030
:10255000092070470C3C02400348006840F00040EE
:102560000149086070470000103C024030B5024647
:102570000C46092500F034F80546092D19D10E48FE
:10258000006820F440700C4908600846006840F478
:10259000007008600846006840F0010008601460A0
:1025A00000F01EF805460448006820F001000249CA
:1025B0000860284630BD0000103C02400548006815
:1025C00000F0004028B1044802490C390860034873
:1025D00008607047103C024023016745AB89EFCD8E
:1025E00008B509200090FFF78DFF009002E0FFF78B
:1025F00089FF00909DF800000128F8D09DF80000A8
:1026000008BDF0B50A4600210023002400BF3DE0CC
:10261000012505FA01F3156805EA03049C4234D14B
:1026200005684F000326BE40B543056015794E008E
:10263000B5400668354305601579012D02D015793E
:10264000022D16D185684F000326BE40B543856034
:1026500055794E00B540866835438560456801264A
:102660008E40B5434560456896798E40B6B2354395
:102670004560C5684F000326BE40B543C560D579A7
:102680004E00B540C6683543C560491C1029BFD30C
:10269000F0BDF0B5002300244D07ED0E02FA05F35E
:1026A000CE1000F1200555F826504E07F70E0F26E4
:1026B000BE40B543CF1000F1200646F82750CE109B
:1026C00000F1200555F8265045EA0304CE1000F12C
:1026D000200545F82640F0BD0246002013690B4056
:1026E0000BB1012000E00020704741837047018357
:1026F0007047000017B500210023BDF800004FF619
:10270000FF74A04203D14348007801431BE0BDF8A9
:102710000000B0F57A7F03D13E484078014312E0D3
:10272000BDF80000B0F5FA7F03D13A488078014344
:1027300009E0BDF80000142803D13648C0780143F1
:1027400001E000201EBD9DF8050038B99DF802008B
:10275000012803D130480078014318E09DF80500B6
:1027600038B99DF8020020B92B4840780143012375
:102770000DE09DF80500012807D19DF8020020B961
:10278000254880780143012301E00020DAE7F3B116
:102790009DF80400012802D09DF8040000B935E03E
:1027A0009DF80400142802D141F008012EE09DF8A4
:1027B0000400052802D141F0400127E09DF8040003
:1027C000642802D141F0480120E00020BAE79DF8DA
:1027D0000400012802D09DF8040000B916E09DF81D
:1027E0000400052802D141F008010FE09DF8040023
:1027F000142802D141F0480108E09DF80400642843
:1028000002D141F0480101E000209BE71160012066
:1028100098E7000003010020000100200FB502210D
:102820009DF8060000F0010008B141F080019DF81C
:10283000050000B91BE09DF80500012802D141F018
:10284000080114E09DF80500022804D1106840F04A
:10285000004010600BE09DF80500032804D11068CB
:1028600080F00040106002E0002004B000BD9DF840
:102870000200012802D141F0400105E09DF802006C
:1028800000B901E00020F0E79DF80400012800D124
:1028900008E09DF80400052802D141F0200101E084
:1028A0000020E2E719700120DFE70000F7B50425FA
:1028B00003269DF80470012F01D1022501261D4831
:1028C0009DF800700FB92F4600E0374639469DF855
:1028D00003707F1EC7EB0717DFF85CC0674401EB8E
:1028E000410C17F80C707F1F17709DF803707F1E46
:1028F000C7EB0717DFF840C0674401EB410C6744A2
:10290000BB789DF803707F1EC7EB0717DFF828C060
:10291000674401EB410C67447C7840EA036040EA7D
:102920000440BDF8017038431778012F00D100BF73
:10293000FEBD000000003010C400002000487047B9
:102940000000002002480349086000BFFEE70000C5
:102950000400FA050CED00E0002111E00846082211
:1029600008E000F001031BB1074B83EA500000E0D0
:102970004008521E002AF4DC044B43F82100491C95
:10298000FF29EBDD704700002083B8EDB002002086
:1029900030B502460B464FF0FF31002008E0CCB2C4
:1029A000155C6C40044D55F8244084EA1121401C0C
:1029B0009842F4D3C84330BDB002002030B503467E
:1029C00009B9012030BD084601EBD0725210A1EBCD
:1029D00042020AB10020F5E7084601EBD072C2F3CB
:1029E0004F04002209E0985CC043C0B215195D5D38
:1029F000A84201D00020E5E7521CA242F3DB0120EF
:102A0000E0E72DE9F04381460C4615461E4614B911
:102A10000120BDE8F083012704F0FF0856B12046ED
:102A200004EBD071C1F3470821464846FFF7C6FFC3
:102A300000B90027A84500D000273846E9E710B5BF
:102A40000246002004E0135CDB4344181355401C8D
:102A50008842F8DB10BD10B502460023002003E0D9
:102A6000145C1C44A3B2401C8842F9D3184610BD24
:102A700010B50446012C04D104210448FFF737FEA9
:102A800003E004210148FFF730FE10BD00100240B2
:102A90001CB50121022000F011FE4FF4C05000903F
:102AA00001208DF8040000208DF8060003208DF829
:102AB000050001208DF8070069460B48FFF7A1FDCE
:102AC00001200A4908600A49C1F8AC0201210948FD
:102AD000FFF70DFE4FF400510348FFF708FE0421F5
:102AE0000548FFF704FE1CBD00040240B0824042CE
:102AF00000804042000C02400000024070B50446D5
:102B00001548006820F44000134908600846006832
:102B100040F480000860002010490860002517E09C
:102B2000E0090E49091F08606006040E022001F04A
:102B300083FA01200A49C1F8B002022001F07CFAB0
:102B4000002006490860022001F076FA681CC5B230
:102B5000082DE5DB70BD000000040240B082404259
:102B60000080404210B50F48006820F440000D4935
:102B700008600846006840F48000086001200A49A7
:102B800008600A49C1F8B002042001F055FA00209B
:102B900005490860042001F04FFA00200349C1F8FC
:102BA000B00210BD00040240AC82404200804042AE
:102BB00010B50F48006820F440000D490860084631
:102BC000006840F48000086000200A4908600A4953
:102BD000C1F8AC02042001F02FFA01200549086079
:102BE0000549C1F8AC02042001F026FA10BD00002E
:102BF00000040240B08240420080404210B50024F0
:102C00001348006820F44000114908600846006835
:102C1000086001200F49086001F00EFA01200E49FA
:102C2000C1F8B00201F008FA07E0601CC4B2FA2C47
:102C300003DDFFF7BDFF012010BD064880380068A6
:102C40000028F2D10349091D086000BFF4E7000025
:102C500000040240AC8240420080404210B5002097
:102C60000F4908600F48006820F440400D49086093
:102C70000846006840F48040086000200A49C1F816
:102C80009C020A2001F0D8F90120054908600A20B9
:102C900001F0D2F900200449C1F8980210BD0000EB
:102CA0009882404200040240008040421CB501214D
:102CB000022000F003FDE020009001208DF80400C8
:102CC00000208DF8060003208DF8050000208DF807
:102CD000070069460948FFF794FC0020084908608E
:102CE0000A2001F0A9F901200649C1F8940204491B
:102CF000091D08600349C1F89C021CBD0004024084
:102D0000948240420080404210B500200F49086084
:102D10000F48006820F440400D49086008460068EC
:102D200040F48040086001200A49C1F89C020A2052
:102D300001F082F90120054908600A2001F07CF9C0
:102D400000200449C1F8980210BD0000988240425A
:102D5000000402400080404270B505460024164839
:102D6000006820F440401449086008460068086084
:102D7000002616E00020114908600A2001F05CF9E5
:102D800001200F49C1F898026006040E0B487C38F8
:102D9000006808B1601CC4B20A2001F04DF9701C33
:102DA000C6B2082EE6DB15B9FFF7AEFF01E0FFF76C
:102DB00055FF204670BD000000040240988240424A
:102DC0000080404270B504461548006820F4404039
:102DD000134908600846006840F4804008600020FD
:102DE00010490860002517E0E0090E49091D086038
:102DF0006006040E0A2001F01FF901200A49C1F8FB
:102E000098020A2001F018F90020064908600A20FB
:102E100001F012F9681CC5B2082DE5DB70BD000099
:102E200000040240988240420080404210B50F48A2
:102E3000006820F440400D4908600846006840F4EE
:102E40008040086001200A4908600A49C1F89802D8
:102E50000A2001F0F1F80020054908600A2001F07D
:102E6000EBF800200349C1F8980210BD00040240AD
:102E70009C8240420080404210B5022001F0DCF804
:102E80001048006820F440400E4908600846006879
:102E900040F48040086000200B4908600B49C1F8ED
:102EA0009C020A2001F0C8F80120074908600520AB
:102EB00001F0C2F801200549C1F89C020A2001F086
:102EC000BBF810BD0004024098824042008040429E
:102ED00010B500241148006820F440400F490860F4
:102EE0000846006808600A2001F0A6F801200C4995
:102EF00008600A2001F0A0F807E0601CC4B2FA2CB8
:102F000003DDFFF7B9FF012010BD05487C380068DC
:102F10000028F2D10249086000BFF5E70004024032
:102F20009882404210B500F001F810BD4AF6AA2080
:102F300001490860704700000030004070B5054648
:102F40000E46002410E02A5D02F0010104F1260281
:102F5000D0B200F017F82A5D52105100621CD0B2B6
:102F600000F010F8601CC4B2B442ECDB00F001F8D1
:102F700070BD10B50121252000F004F8142001F0E7
:102F80005BF810BD70B506460D460024102000F019
:102F9000EEF8C82001F050F8FFF748FF7820FFF75F
:102FA00011FFFFF795FF044604B110E03046FFF72C
:102FB00009FFFFF78DFF044604B108E02846FFF73C
:102FC00001FFFFF785FF044604B100E000BFFFF7F3
:102FD00053FFC82001F030F870BD000010B54FF469
:102FE000A06000F067F80121022000F067FBA82034
:102FF00000F0E4FF4FF4E13001F012F9FDF786FB39
:10300000FEF7F8FD00F074F9FDF708FBFFF7ACF8E8
:10301000002000F021FB01200149087010BD0000D4
:10302000AA00002002480349086000BFFEE7000034
:103030000400FA050CED00E07047000070B50021B7
:1030400000230F22C4781CB3174C246804F4E064F6
:10305000C4F5E064C4F30721C1F10404E3B20A41FA
:1030600044789C40E1B28478144021430C07210E3F
:103070000E4C05786155047804F01F050124AC401E
:1030800005786D11AD0005F1E025C5F8004109E0B6
:10309000047804F01F050124AC40054D0678761134
:1030A00045F8264070BD00000CED00E000E400E0B3
:1030B00080E100E002490143024A116070470000CC
:1030C0000000FA050CED00E070B582240325FFF73F
:1030D000ADFE2046FFF776FEFFF7FAFE00B10EE0E8
:1030E0002846FFF76FFEFFF7F3FE00B107E0002070
:1030F000FFF768FEFFF7ECFE00B100E000BFFFF74E
:10310000BBFE70BD70B5044682250126FFF78EFE1A
:103110002846FFF757FEFFF7DBFE00B110E0304610
:10312000FFF750FEFFF7D4FE00B109E004F0010103
:10313000881CFFF747FEFFF7CBFE00B100E000BFA1
:10314000FFF79AFE70BD70B50024FFF76FFEE12512
:103150002846FFF737FEFFF7BBFE0020FFF7FCFD18
:103160000446FFF7D1FDFFF787FE204670BD70B51E
:103170000446FFF75BFEE0252846FFF723FEFFF736
:10318000A7FE00B107E02046FFF71CFEFFF7A0FEF8
:1031900000B100E000BFFFF76FFE70BD70472DE982
:1031A000F05F04460E46207800F00107207800F01A
:1031B0000208207800F00409207800F0080A20783E
:1031C00000F0100B002537B101252846FFF7CFFF8F
:1031D000012000F011FFB8F1000F06D002252846AB
:1031E000FFF7C5FF012000F007FFB9F1000F06D07F
:1031F00004252846FFF7BBFF012000F0FDFEBAF1D1
:10320000000F06D008252846FFF7B1FF012000F087
:10321000F3FEBBF1000F06D010252846FFF7A7FFED
:10322000012000F0E9FEFFF78EFFA84202D0002047
:10323000BDE8F09F35B1642231460020FDF757F913
:103240006420F5E70020F3E72DE9F05F04460E4621
:10325000207800F00107207800F00208207800F0C4
:103260000409207800F0080A207800F0100B0025EF
:1032700037B101252846FFF77AFF012000F0BCFE98
:10328000B8F1000F06D002252846FFF770FF012095
:1032900000F0B2FEB9F1000F06D004252846FFF772
:1032A00066FF012000F0A8FEBAF1000F06D0082545
:1032B0002846FFF75CFF012000F09EFEBBF1000FE7
:1032C00006D010252846FFF752FF012000F094FE9B
:1032D000FFF739FFA84202D00020BDE8F09F2DB1D2
:1032E000642231460020FDF750F9F6E70020F4E7AC
:1032F0001CB501210D2000F0E1F9542000900020C0
:103300008DF8040001208DF8060003208DF80500DB
:1033100000208DF8070069460F48FFF772F94FF457
:10332000A050009069460D48FFF76BF94FF44070CC
:10333000009001208DF8070069460848FFF761F901
:1033400069460748FFF75DF94FF400400090694671
:103350000148FFF756F91CBD000C02400000024076
:10336000000802402DE9F04740212748FFF7B4F953
:10337000054610212448FFF7AFF9064604212248EC
:10338000FFF7AAF907464FF480512048FFF7A4F948
:1033900080464FF480611D48FFF79EF981461C4826
:1033A000007818B9002501201949087019480078DB
:1033B00018B900260120174908701748007818B975
:1033C00000270120144908701448007820B94FF0F4
:1033D00000080120114908701148007820B94FF009
:1033E000000901200E49087045F0E00040EA46005F
:1033F00040EA870040EAC80040EA0910C043C4B26E
:103400002046BDE8F0870000000C024000000240AA
:10341000A5000020A6000020A7000020A800002092
:10342000A90000202DE9F0474FF400717748FFF71D
:1034300053F904464FF480717448FFF74DF905467F
:103440004FF400717248FFF747F906464FF4807158
:103450006F48FFF741F907464FF400416D48FFF709
:103460003BF9804644F0E00040EA450040EA86002F
:1034700040EAC70040EA0810C04300F0FF094FF4DB
:1034800000716248FFF728F963490978884216D02D
:103490004FF400715D48FFF71FF980B91E2000F05E
:1034A000ABFD4FF400715948FFF716F938B9012008
:1034B000FFF75DFE012000F09FFDFFF705FE4FF4D2
:1034C00080715248FFF708F954490978884216D0AC
:1034D0004FF480714D48FFF7FFF880B91E2000F0CF
:1034E0008BFD4FF480714948FFF7F6F838B9022098
:1034F000FFF73DFE012000F07FFDFFF7E5FD4FF4F3
:1035000000714348FFF7E8F845490978884216D02A
:103510004FF400713E48FFF7DFF880B91E2000F03D
:103520006BFD4FF400713A48FFF7D6F838B9042024
:10353000FFF71DFE012000F05FFDFFF7C5FD4FF412
:1035400080713348FFF7C8F836490978884216D0A9
:103550004FF480712E48FFF7BFF880B91E2000F0AD
:103560004BFD4FF480712A48FFF7B6F838B90820B0
:10357000FFF7FDFD012000F03FFDFFF7A5FD4FF433
:1035800000412448FFF7A8F827490978884216D057
:103590004FF400411F48FFF79FF880B91E2000F04C
:1035A0002BFD4FF400411B48FFF796F838B9102067
:1035B000FFF7DDFD012000F01FFDFFF785FD4FF453
:1035C00000711248FFF788F8134908704FF48071B2
:1035D0000E48FFF781F8114908704FF400710C484C
:1035E000FFF77AF80E4908704FF480710848FFF72A
:1035F00073F80C4908704FF400410648FFF76CF867
:10360000094908704846BDE8F08700000000024004
:1036100000080240000C0240A0000020A100002091
:10362000A2000020A3000020A400002070B50446E2
:103630000D46052C00DC04B970BD601EC4B201212A
:10364000A140C8B2FFF793FD012000F0D5FC284649
:10365000FFF758FD00BFEFE72DE9F047044604F0FF
:103660000105C4F34006C4F38007C4F3C008C4F3E3
:10367000001929460120FFF7D9FF012000F0BCFC0A
:1036800031460220FFF7D2FF012000F0B5FC394699
:103690000320FFF7CBFF012000F0AEFC41460420E1
:1036A000FFF7C4FF012000F0A7FC49460520FFF703
:1036B000BDFF012000F0A0FCBDE8F08729B1064A5B
:1036C00012680243044B1A6004E0034A1268824302
:1036D000014B1A60704700003038024029B1064A99
:1036E00012680243044B1A6004E0034A12688243E2
:1036F000014B1A607047000044380240F0B50021C9
:1037000000220024022500260223324F3F6807F0E2
:103710000C0121B1042905D0082937D105E02E4F2D
:10372000076036E02D4F076033E02A4F3F1F3F68A8
:10373000C7F38056274F3F1F3F6807F03F036EB126
:10374000264FB7FBF3F7DFF88CC0ACF1040CDCF8C4
:1037500000C0CCF3881C07FB0CF40CE01E4FB7FB39
:10376000F3F7DFF870C0ACF1040CDCF800C0CCF368
:10377000881C07FB0CF4174F3F1F3F68C7F3014736
:103780007F1C7D00B4FBF5F7076002E0124F076075
:1037900000BF00BF0F4F3F6807F0F0010909104F4D
:1037A0007A5C0768D74047600A4F3F6807F4E051EA
:1037B000890A0B4F7A5C4768D7408760054F3F689E
:1037C00007F46041490B064F7A5C4768D740C760F1
:1037D000F0BD0000083802400024F40000127A0016
:1037E0000701002001461C48814201D20020704799
:1037F0001A48814201D20820F9E71948814201D2D2
:103800001020F4E71748814201D21820EFE716484C
:10381000814201D22020EAE71448814201D22820C7
:10382000E5E71348814201D23020E0E711488142A8
:1038300001D23820DBE71048814201D24020D6E790
:103840000E48814201D24820D1E70D48814201D281
:103850005020CCE75820CAE700400008008000084C
:1038600000C0000800000108000002080000040871
:10387000000006080000080800000A0800000C0804
:1038800000000E0830B503460C461546002206E03F
:10389000184600F007F844F822001B1D521CAA42EB
:1038A000F6D330BD01460868704700002DE9F047A7
:1038B00004460E4617464FF009080025A946B4F104
:1038C000006F02D304F0030008B1BDE8F087FEF7F3
:1038D00075FE0020FEF7C0FD254604EB8709194858
:1038E000854218D214E02846FFF7DCFF401C70B177
:1038F000F120FEF7ABFD2846FFF774FF8246022158
:10390000FEF7BCFD8046B8F1090F01D002E02D1D85
:103910004D45E8D300BFB8F1090F0CD108E02046AF
:103920003168FEF723FE092800D003E0241D361D70
:103930004C45F4D300BF0120FEF78EFDFEF70CFED0
:1039400000BFC2E70000FF1F7047000030B5002233
:103950008B071C0F0F2303FA04F20B4B8C1053F848
:1039600024309343084C8D1044F8253023468C10A6
:1039700053F824308C07240F00FA04F42343024C3C
:103980008D1044F8253030BD083801400CB50020BA
:10399000019000903448006840F48030324908605B
:1039A00000BF3148006800F4003000900198401CCE
:1039B0000190009818B90198B0F5A04FF1D12A48AC
:1039C000006800F4003010B10120009001E00020F8
:1039D00000900098012846D123484030006840F00C
:1039E00080502149403108602048006840F4404040
:1039F0001E4908601C48083000681B4908310860EF
:103A00000846006840F4004008600846006840F43A
:103A1000A05008601648091F0860081F006840F0A1
:103A20008070091F086000BF0F48006800F0007038
:103A30000028F9D040F205700E4908600A480830A5
:103A4000006820F003000849083108600846006853
:103A500040F00200086000BF03480830006800F032
:103A60000C000828F8D10CBD00380240007000405E
:103A700008544007003C0240042808D14FF0E021E0
:103A8000096941F004014FF0E022116107E04FF0B5
:103A9000E021096921F004014FF0E0221161704733
:103AA0007047000010B51548006840F470001349D5
:103AB00008601348006840F00100114908600020C8
:103AC0000F49083108600E4800680E4908400C494B
:103AD00008600D48091D0860081F006820F4802058
:103AE000091F0860002006490C310860FFF74EFFEF
:103AF0004FF0006001498039086010BD88ED00E09A
:103B000000380240FFFFF6FE1030002410B50121FE
:103B1000054800F010F8012801D10449087001217E
:103B2000014800F005F810BD00040040AB00002083
:103B3000CA430282704730B50246002000230024A9
:103B4000158A05EA0103958905EA010413B10CB150
:103B5000012000E0002030BD70B504460D46FFF79F
:103B600061FC00B21E490880FFF7FCFB00B21D4952
:103B70000880012C10D11C48B0F900001849B1F997
:103B80000010884208D11948B0F900001549B1F970
:103B90000010884200D170BD1148B0F900001249F0
:103BA00008801048B0F900001049088002260C482F
:103BB00000780F4908700B48007848702A46314653
:103BC000312000F013F90648B0F9000006490880DA
:103BD0000448B0F900000549088000BFDBE7000099
:103BE000A0020020A2020020A4020020A6020020C1
:103BF000B8460020002005E04FF6FF710A4A22F87F
:103C00001010401C1428F7DB0020084908700849F0
:103C10000870084908600849087008490880084980
:103C2000088008490880704738570020AD00002000
:103C3000AC000020B0000020B4000020B60000203E
:103C4000B8000020BA0000205E49098801F0200178
:103C500021B15C49091D0988C8B200E070475A4982
:103C600009780A297BD2DFE801F00517232F353BBD
:103C70004E52616D55280ED10121544A1170544A9B
:103C800011800021534A118001214F4A117052497D
:103C90000988524A118063E0AA2803D102214A4AC6
:103CA000117004E00021494A1170474A117057E031
:103CB000BB2803D10321444A117004E00021434A88
:103CC0001170414A11704BE004213F4A1170414983
:103CD000088045E005213C4A11703E4908803FE0DC
:103CE0000621394A11703B49098841EA0021394AC5
:103CF00011800021364A11803649098811B90821FE
:103D0000314A11702CE007212F4A117000BF304951
:103D10000988491C2E4A1180114609882D4A1288AB
:103D2000914202DB0821284A117019E00D2805D0C4
:103D30000021264A1170244A117002E00921224A0A
:103D400011700DE00A2806D00021204A11701E4A89
:103D5000117003E003E00A211B4A117000E000BF6C
:103D600000BF1A49097881B11B490A680968491CD2
:103D7000194B19601A4988541946096844F2080217
:103D8000914202D300211A4611600F4909780A298D
:103D900015D112490988134A134B1B7822F81310C6
:103DA00011490978491C142291FBF2F302FB13110B
:103DB0000D4A11700021054A1170034A117000BFAD
:103DC0004CE7000000140140AD000020B4000020CA
:103DD000BA000020B8000020B0000020B60000208B
:103DE000B006002038570020AC0000202DE9F04735
:103DF00081460C461646274626B1A1B21048FEF76A
:103E00001EFE7F000F4B3A460D494846FDF76EFCFB
:103E1000804640210C4800F019F800250CE00948C4
:103E2000415D094800F0C4F800BF4021064800F099
:103E300022F80128F9D16D1C4545F0DBBDE8F0877B
:103E4000B8460020B84E00200014014001F4007272
:103E5000B2F5007F00D100BFCA430280704721B194
:103E6000828942F40052828104E082894DF6FF7318
:103E70001A408281704702460020B1F5007F00D1D0
:103E800000BF13880B400BB1012000E000207047F9
:103E9000F0B50346002400260025002040F66A17EE
:103EA000B94200D100BF1846C1F3421401F01F0609
:103EB000012707FA06F5012C01D10C3004E0022C91
:103EC00001D1103000E014301AB107682F430760A9
:103ED00002E00768AF430760F0BD00002DE9FF472F
:103EE00005460E460024A14600BFA046B08900B199
:103EF00000BF2C8A24F44054F08804432C82AC89FF
:103F000041F20C608443B0883189084371890843C9
:103F10000443AC81AC8A24F44074B0890443AC827D
:103F20006846FFF7EBFB2048854202D01F488542D8
:103F300002D1DDF80C9001E0DDF80890A88900F4CA
:103F4000004040B109EBC90000EB0910316849009D
:103F5000B0FBF1F707E009EBC90000EB091031688D
:103F60008900B0FBF1F76420B7FBF0F004012009F1
:103F7000642101FB1078A88900F4004040B1322090
:103F800000EBC800B0FBF1F000F00700044308E0CC
:103F9000322000EB08106421B0FBF1F000F00F00BC
:103FA00004432C81BDE8FF8700100140001401404C
:103FB000C1F308028280704700BFFEE710B50446D7
:103FC0006FF00400FFF758FDE11704EB5171C1F3E6
:103FD000C701074A11701046007800EB4001C1EBA1
:103FE000C0104FF6FF7101EAC0000249088010BD01
:103FF0009C0000209E00002070B504464FF407701E
:1040000094FBF0F0C6B24FF4077094FBF0F100FBA4
:10401000114085B204B970BD05E04FF4077000F09F
:1040200031F8701EC6B2002EF7D115B1284600F047
:1040300029F800BFEFE700000146114A12784A4311
:104040004FF0E0235A6100229A611A46126942F049
:1040500001021A6100BF4FF0E022106900F0010276
:104060001AB100F48032002AF5D04FF0E022126934
:1040700022F001024FF0E0231A6100229A6170479A
:104080009C0000200146114A12884A434FF0E02369
:104090005A6100229A611A46126942F001021A61BD
:1040A00000BF4FF0E022106900F001021AB100F4E5
:1040B0008032002AF5D04FF0E022126922F001028E
:1040C0004FF0E0231A6100229A6170479E000020A1
:1040D00010B50446282221460148FFF7D3FB10BD46
:1040E0000000010810B50446282221460148FFF7C8
:1040F000DDFB10BD0000010800B5A9B06846FFF760
:10410000E7FF4FF0FF30CDF882006846FFF7EAFF87
:104110000A20FFF771FF29B000BD0000FEF75EFF27
:10412000FEF71AFC0024FDF747FDFDF745FD0121D0
:104130002948FDF799FC02212748FDF795FC1F2728
:10414000A04600250CE0681CC2B239460420FDF7E9
:1041500073FE681CC2B241460520FDF76DFE6D1C62
:10416000042DF0DBFDF764FB00260CE0642094FBDB
:10417000F0F100FB114008B9FEF7D4FE641C3220B8
:10418000FFF75AFF761CB6F57A7FEFDB0024FDF7C8
:104190004FFB1FE03220FFF74FFF642094FBF0F14C
:1041A00000FB114008B9FEF7BDFEFCF7CDFAFDF7A4
:1041B000BDFA0A480078012800D10BE0B4F57A7FF7
:1041C00006DB01210846FFF7C7FCFDF7F5FC0024DC
:1041D000641C00BFDEE70000FF7F20008400002099
:1041E0000D48006840F480200B4908600A481038E8
:1041F000006840F0100008491039086003200121D0
:104200008140064A430942F8231000BFBFF34F8F95
:10421000BFF36F8F7047000024ED00E000E200E084
:1042200010B588B0044601210420FFF747FA0121A8
:104230002020FFF753FA082206212548FEF729FA25
:10424000082207212248FEF724FAC0200690022007
:104250008DF81C008DF81D0000208DF81E00012037
:104260008DF81F0006A91A48FEF7CBF9029400202A
:10427000ADF80C00ADF80E00ADF81000ADF814006C
:104280000C20ADF8120002A91248FFF727FE012109
:104290001048FFF7E4FD40210E48FFF7D7FD01224B
:1042A00040F225510B48FFF7F3FD47208DF804003D
:1042B00002208DF8050003208DF8060001208DF8FE
:1042C000070001A8FEF7BAFEFFF794FC08B010BD86
:1042D00000080240001401404FF04070E1EE100A67
:1042E000704700000443000800000020B0020000F6
:1042F000C401000870440008B0020020687D00007E
:104300002002000811130A08801732303233303986
:1043100031313130333233357A68616F796F6E679E
:1043200078104A6948654D736F37303030583264C1
:104330003518810026394170702C526561645465CE
:104340006D70657261747572652C6E6577416E6112
:104350006C6F67436F6D6D4D6F64657A0101011A73
:104360001506050806280B080604080602080607B5
:10437000080F1010060806030806010807030A07BD
:10438000050A07280A0A07040A07020A07070F1284
:1043900008200D0C08040C08020C08070C10203C27
:1043A0000501036B2C020304041943D209180832D7
:1043B0003032322D3031033D2030303A0311298F15
:1043C00013F90B2A080932021B210C0C31294A4B24
:1043D0000D0D0C2A04554A0E2432051A390C29C831
:1043E00032062A710C3132075AB52432155AE518B3
:1043F0001997114B430F4832215A5B0C32225A5DF8
:104400000C32234B7D103032291AD10C4132304B03
:1044100035115432315AA90C32322AC10C3132339F
:104420001AD90C299032344B4912482A4054590C5D
:1044300032415AFD0C32424B85130C32434B1D1452
:104440000C2A4818590C32505AB90C32C14B61151C
:104450006C32E05A750C32E15A8D0C32E31A950C2D
:10446000293032E44B71161801101AFF0181000047
:040000050800018965
:00000001FF
